:10000000000000308A006D280F39A8000310A80DE9
:10001000A80D1F08C039280401389F0032302E2057
:100020009F149F1811281E08AB0083161E08831208
:10003000AA00692883178001840AFF3E031D1B283C
:100040006928A501A400FF30A407031CA507031C11
:1000500069280330A300E3302F202328A301F43EB6
:10006000A200A309FE30031C3828A2070318352874
:10007000A2070000A30F3528000022183F282218ED
:1000800041280800A701A6011030A800230DA60DE5
:10009000A70D2408A6022508031C250FA702031894
:1000A00058282408A60725080318250FA7070310BA
:1000B000A20DA30DA80B462822080800A200A31B2E
:1000C000632022086928A209A309A20A0319A30A26
:1000D000080083138312031308008301C0309F00BC
:1000E000713083168F008312850186018701831684
:1000F000811701308500860187010317880083126C
:1001000003139F00803083169F0083128A110A1206
:100110006A29340836028A110A12031D9528330809
:1001200035028A110A12031969298312031333084D
:100130003502A2003408031C013E3602A3008A01E6
:100140005F20A0002308A100033021028A110A12B7
:10015000031CB4288A110A12031DB628E9302002B4
:100160008A110A120318B6280301031D01308312F5
:100170000313B000B6088A110A12031DC5281030F7
:1001800035028A110A12031CC7280301031D01301E
:1001900083120313B0048A110A120319D2288A1198
:1001A0000A12122933083502A2003408031C013E4A
:1001B0003602A3008A015F20A0002308A100A10845
:1001C0008A110A12031DEA28103020028A110A122D
:1001D000031C192983120313340CAB00330CAA003F
:1001E000AB0CAA0CAB0CAA0CAB0CAA0C0F30AB05D9
:1001F0002A083302B3002B08031C013E3402B4006A
:10020000360CAB00350CAA00AB0CAA0CAB0CAA0C3C
:10021000AB0CAA0C0F30AB052A08B3072B08031848
:10022000013EB4073608B4003508B3008A110A123B
:1002300065293408AB003308AA003408AD00330840
:10024000AC00AF011030AE000310AF0CAE0C0310C9
:10025000AF0CAE0C2D08A3002C08A2002F08A5009F
:100260002E08A4008A014220AC002308AD002C080F
:100270002A02B3002D08031C013E2B02B4003408EF
:10028000AB003308AA003608AD003508AC00AF015A
:100290001030AE000310AF0CAE0C0310AF0CAE0C60
:1002A0002D08A3002C08A2002F08A5002E08A400EA
:1002B0008A014220AC002308AD002A082C07B300B5
:1002C0002B080318013E2D07B4003408B60033088C
:1002D000B500080064308A0121202030840060309D
:1002E0008A011B20A030840050308A011B2010306E
:1002F000840060308A011A209030840060308A01C6
:100300001A2083168711831287118316071183120F
:100310000711831687108312871083160710831224
:100320000710831605138312051383168513831292
:100330008513831685128312851283160512831284
:1003400005128316851183128511831605118312F8
:100350000511831685108312851083168613831268
:1003600086138316071283120712831687128312CD
:10037000871283160713831207138316071083123D
:100380000710831606108312061083168610831238
:1003900086108316061183120611831686118312A6
:1003A0008611831606128312061283168612831292
:1003B0008612831606138312061300308A01042066
:1003C000B1002B08B2003208B6003108B5008A012E
:1003D00089203608B2003508B100B2088A110A1225
:1003E000031DFE29143031028A110A120318FE2956
:1003F0008501860187018A110A12D52CB2088A115B
:100400000A12031D092A143031028A110A12031C30
:100410001D2A83120313B2088A110A12031D1D2A12
:10042000283031028A110A1203181D2A850186011B
:10043000083087008A110A12D52CB2088A110A12D4
:10044000031D282A283031028A110A12031C3C2A73
:1004500083120313B2088A110A12031D3C2A3C308E
:1004600031028A110A1203183C2A850186010C30D8
:1004700087008A110A12D52CB2088A110A12031DAC
:10048000472A3C3031028A110A12031C5B2A83126C
:100490000313B2088A110A12031D5B2A503031027D
:1004A0008A110A1203185B2A850186010E30870023
:1004B0008A110A12D52CB2088A110A12031D662A63
:1004C000503031028A110A12031C7A2A8312031354
:1004D000B2088A110A12031D7A2A643031028A1185
:1004E0000A1203187A2A850186010F3087008A11C3
:1004F0000A12D52CB2088A110A12031D852A64300B
:1005000031028A110A12031C9A2A83120313B208B9
:100510008A110A12031D9A2A783031028A110A12AE
:1005200003189A2A4030850086010F3087008A110F
:100530000A12D52CB2088A110A12031DA52A783096
:1005400031028A110A12031CBA2A83120313B20859
:100550008A110A12031DBA2A8C3031028A110A123A
:100560000318BA2AC030850086010F3087008A112F
:100570000A12D52CB2088A110A12031DC52A8C3022
:1005800031028A110A12031CDA2A83120313B208F9
:100590008A110A12031DDA2AA03031028A110A12C6
:1005A0000318DA2AE030850086010F3087008A11AF
:1005B0000A12D52CB2088A110A12031DE52AA030AE
:1005C00031028A110A12031CFA2A83120313B20899
:1005D0008A110A12031DFA2AB43031028A110A1252
:1005E0000318FA2AF030850086010F3087008A113F
:1005F0000A12D52CB2088A110A12031D052BB43039
:1006000031028A110A12031C1A2B83120313B20837
:100610008A110A12031D1A2BC83031028A110A12DC
:1006200003181A2BF830850086010F3087008A11D5
:100630000A12D52CB2088A110A12031D252BC830C4
:1006400031028A110A12031C3A2B83120313B208D7
:100650008A110A12031D3A2BDC3031028A110A1268
:1006600003183A2BFC30850086010F3087008A1171
:100670000A12D52CB2088A110A12031D452BDC3050
:1006800031028A110A12031C5A2B83120313B20877
:100690008A110A12031D5A2BF03031028A110A12F4
:1006A00003185A2BFE30850086010F3087008A110F
:1006B0000A12D52CB2088A110A12031D652BF030DC
:1006C00031028A110A12031C822B01308312031398
:1006D00032028A110A12031C772B8A110A12031D97
:1006E000822B043031028A110A120318822BFE3049
:1006F000831203138500803086000F3087008A1133
:100700000A12D52C013032028A110A12031CAF2BB7
:100710008A110A12031D922B043031028A110A1227
:10072000031CAF2B01308312031332028A110A1209
:10073000031CA42B8A110A12031DAF2B183031029F
:100740008A110A120318AF2BFE308312031385009F
:10075000803086001F3087008A110A12D52C0130A4
:1007600032028A110A12031CDC2B8A110A12031DA1
:10077000BF2B183031028A110A12031CDC2B013006
:100780008312031332028A110A12031CD12B8A111D
:100790000A12031DDC2B2C3031028A110A120318B5
:1007A000DC2BFE30831203138500803086003F303F
:1007B00087008A110A12D52C013032028A110A12DE
:1007C000031C092C8A110A12031DEC2B2C30310258
:1007D0008A110A12031C092C0130831203133202FE
:1007E0008A110A12031CFE2B8A110A12031D092CFE
:1007F000403031028A110A120318092CFE3083128C
:1008000003138500803086007F3087008A110A122A
:10081000D52C013032028A110A12031C362C8A119F
:100820000A12031D192C403031028A110A12031CCE
:10083000362C01308312031332028A110A12031C70
:100840002B2C8A110A12031D362C543031028A11C6
:100850000A120318362CFE308312031385008030F1
:100860008600FF3087008A110A12D52C013032022F
:100870008A110A12031C632C8A110A12031D462CCA
:10088000543031028A110A12031C632C0130831286
:10089000031332028A110A12031C582C8A110A12FD
:1008A000031D632C683031028A110A120318632C6D
:1008B000FE3083120313850081308600FF308700ED
:1008C0008A110A12D52C013032028A110A12031C35
:1008D000902C8A110A12031D732C683031028A1180
:1008E0000A12031C902C01308312031332028A1166
:1008F0000A12031C852C8A110A12031D902C7C30CD
:1009000031028A110A120318902CFE30831203134D
:10091000850083308600FF3087008A110A12D52CAB
:10092000013032028A110A12031CBD2C8A110A12EC
:10093000031DA02C7C3031028A110A12031CBD2C2D
:1009400001308312031332028A110A12031CB22CE3
:100950008A110A12031DBD2C903031028A110A122D
:100960000318BD2CFE3083120313850087308600E8
:10097000FF3087008A110A12D52C013032028A1109
:100980000A12031CD52C8A110A12031DCD2C91309A
:1009900031028A110A12031CD52CFE308312031374
:1009A00085008F308600FF3087008A01DD298A01AB
:0209B000D72C42
:02400E00A42CE0
:02401000FF3F70
:00000001FF
